:0600000075817F0200265D
:100023000201F67545007547017546007544007574
:1000330043007590FF1201E3753400753500752E8A
:1000430000752F007530007531007532007533006F
:10005300D2B2C204D208D207D205D209C20DD2123B
:10006300754877C20CD20BD20AC20E7400900010EE
:10007300F0900011F0900012F0900013F090001433
:10008300F01212101212451202D61202D620B2FD3D
:100093001201291202EAE53FB400061200B302007E
:1000A30096B401061200E20200961200F6020096D0
:1000B30030071420B2FD7452120210745812021049
:1000C300120129C207D20520920C12011630050530
:1000D3001201B3C2052220050512019ED20522306A
:1000E3000805120AAFC208209206120A88C2052226
:1000F300D20522300908120AAF754600C209120A56
:1001030076300C0C120B65120B9FC205121245229E
:10011300D20522120EAA1209A2120FF112111F12F6
:100123000CC5120E7C22745C120210743012021081
:1001330012019E7438120210744A120210743012A3
:100143000210744E12021012100F74311202107446
:1001530034120210744A12021074311202107435F0
:10016300120210744E1202107431120210743512FE
:100173000210744A12021074311202107435120202
:1001830010744E1202107436120210744A120210C6
:100193007430120210744E120210227437120210BD
:1001A300744A1202107430120210744E120210229A
:1001B3007437120210744A120210747F1201CB12A8
:1001C3000258744E12021022F52E752F007532015B
:1001D300753300782E793212085686820886832278
:1001E300C2AF438780759B1F759AD9759850D2AC5F
:1001F300D2AF22C0D0C0E020980A30990BC299C276
:100203000002020BC298E599D0E0D0D0322093FDD2
:10021300F599D2002000FD2275F00A84AFF075F045
:100223000A842430120210E5F02430120210EF2465
:10023300301202102275F00A84AFF0EF2430F62258
:1002430075F00A84AFF075F00A84E5F02430F6EF18
:10025300243008F622C0E0E8C0E0C2D5AA82AB830E
:100263007C107D271202B660042430D2D57CE87D51
:10027300031202B6700330D5072430120210D2D510
:100283007C647D001202B6700330D507243012025D
:1002930010D2D5EAABF075F00A84700330D505248B
:1002A30030120210E5F08BF02430120210D0E0F887
:1002B300D0E022780008C3EA9CFAEB9DFB50F618C5
:1002C300EA2CFAEB3DFBE822783279FF0000D9FCF7
:1002D300D8F822784B79FF0000D9FCD8F822780AA5
:1002E3007996D9FED8FA22209108753F00D209D217
:1002F3000822309008753F01D209D20722753F02C8
:10030300D207D20822FD90191893FFA3ED93FE2282
:10031300FD9018E893FFA3ED93FE22B5400302037B
:1003230027754600F540B43B0302033440FB020447
:100333002C75F004A490033C7390128C229012C28B
:10034300229012FB2290130D229013112290131569
:10035300229013192290131D229013222290132707
:100363002290132D22901330229013352290133AAA
:1003730022901341229013442290134A2290134C4B
:100383002290135122901355229013582290135CFC
:0E03930022901361229013652290136722902E
:1003A100136F229013792290137E2290138322904F
:1003B10013892290138F2290139A229013A02290D6
:1003C10013A8229013B1229013B7229013BE22904A
:1003D10013C4229013CB229013D1229013DA2290CE
:1003E10013E0229013E4229013E9229013EE22905D
:1003F10013F5229013FD22901409229014122290D9
:100401001417229014242290142A2290143022903E
:1004110014342290143B2290143F229014442290D1
:10042100144A229014572290146322C3943C75F00D
:1004310004A49004377390146922901475229014C7
:100441007C22901482229014872290148A22901484
:10045100902290149A229014A0229014A522901414
:10046100AC229014B0229014B4229014B9229014AA
:10047100C4229014C9229014CE229014D322901435
:10048100DA229014DF229014E4229014E9229014CD
:10049100F3229014F7229014FD2290150222901558
:1004A100052290150B229015142290151A229015F1
:1004B10020229015252290152A2290152F22901581
:1004C10033229015362290153B229015402290152B
:1004D10043229015462290154A2290154D229015DF
:1004E10052229015572290155C2290155F2290158B
:1004F10062229015672290156A2290156D2290153F
:1005010072229015772290157C22901582229015E7
:10051100862290158A229015942290159922901581
:10052100A5229015A522300E07854182854283229E
:1005310012121012127C1205AB75F006A49005423E
:10054100739015AD0205A29015B00205A29015B2E7
:100551000205A29015BA0205A29015C10205A2904A
:1005610015C80205A29015CF0205A29015D4020567
:10057100A29015DB0205A29015E40205A29015E8F0
:100581000205A29015EF0205A29015F50205A290B1
:1005910015FF0205A290160C0205A290161F020576
:1005A100A2858241858342D20E22B40503C2112263
:1005B10040FBD21122300E078541828542832212EF
:1005C100121012127C75F006A49005CE7390162EAF
:1005D10002062E90163802062E90163C02062E9028
:1005E100164602062E90164B02062E901650020653
:1005F1002E90165C02062E90166602062E90166A42
:1006010002062E90167302062E90167702062E9081
:10061100168102062E90168802062E901692020668
:100621002E90169C02062E9016A402062E8582415B
:10063100858342D20E22300E078541828542832274
:1006410012121012127C75F006A490064F739016C8
:10065100A80206AF9016B30206AF9016B80206AF15
:100661009016C30206AF9016C90206AF9016CF02CC
:1006710006AF9016DC0206AF9016E70206AF9016A1
:10068100ED0206AF9016F70206AF9016FC0206AF18
:100691009017070206AF90170F0206AF90171A02C4
:1006A10006AF9017260206AF90172F0206AF85827C
:1006B10041858342D20E22300E07854182854283D5
:1006C1002212121012127C75F006A49006D07390BB
:1006D100173402073090173F020730901744020782
:1006E1003090174902073090174D02073090175488
:1006F10002073090175E02073090176402073090AE
:10070100176802073090176E0207309017740207BE
:0E0711003090177A0207309017800207309060
:10071F00178802073090179002073090179702073B
:10072F0030858241858342D20E22300E0785418269
:10073F008542832212121012127C75F006A49007C4
:10074F00517390179E0207B19017A40207B190172B
:10075F00AE0207B19017BA0207B19017C50207B1E1
:10076F009017CD0207B19017D30207B19017D90296
:10077F0007B19017E50207B19017F00207B1901774
:10078F00FD0207B19018030207B190180B0207B1D1
:10079F009018110207B19018160207B19018220293
:1007AF0007B1858241858342D20E22300E078541E3
:1007BF00828542832212121012127C75F006A490C9
:1007CF0007D273901829020832901831020832901C
:1007DF00183502083290183802083290184402086F
:1007EF003290185002083290185B0208329018634A
:1007FF0002083290186D0208329018710208329078
:10080F00187602083290187C02083290188102087C
:10081F003290188902083290188E02083290189C74
:10082F00020832858241858342D20E22E627F523C4
:10083F000809E637F524782322C3E697F52308093C
:10084F00E697F524782322862387250809862487AF
:10085F00261208DB782822862808862908862A0887
:10086F00862B872509872612087E7823792A2275F9
:10087F002C00752D101208C01208911208B4D52D36
:10088F00F422C3E52A9525E52B9526E52C940050F7
:10089F000122E52A9525F52AE52B9526F52BE52C42
:1008AF009400F52C22B3E52333F523E52433F52407
:1008BF0022C3E52833F528E52933F529E52A33F551
:1008CF002AE52B33F52BE52C33F52C22E523852553
:1008DF00F0A4F52885F029E5248526F0A4F52A85CE
:1008EF00F02BE5248525F0A42529F529E52A35F0F7
:1008FF00F52AE52B3400F52BE5238526F0A42529D1
:10090F00F529E52A35F0F52AE52B3400F52B227A67
:10091F000FC295D294A29633C933C9C294DAF2F8B2
:10092F00D29522D2957A0574E0C294C295339297EC
:10093F00D294DAF512091E8836893753370F22D22F
:10094F00957A0574E8C294C295339297D294DAF5EA
:10095F0012091E8838893953390F22D2957A0574B6
:10096F00F0C294C295339297D294DAF512091E8889
:10097F003A893B533B0F22D2957A0574F8C294C241
:10098F0095339297D294DAF512091E883C893D531C
:10099F003D0F2212093285362E85372F753000759F
:1009AF003100782E75320A753300793212083B8682
:1009BF002E08862F753000753100782E75320A7526
:1009CF003300793212085675325575330179321268
:1009DF000866E675F002A4F5492212093285362E13
:0B09EF0085372F753000753100782E21
:1009FA0075320A753300793212083B862E08862F23
:100A0A00753000753100782E75320A7533007932E7
:100A1A001208567532557533017932120866E61294
:100A2A0011F175F002A4120313EE22120986853C15
:100A3A002E853D2F753000753100782E753214756C
:100A4A003300793212083B862E08862F75300075DE
:100A5A003100782E75320A753300793212085675CC
:100A6A0032557533017932120866E62220920C203B
:100A7A000D08D20CD20DD20AD20B22C20D2220B2FC
:100A8A00FD7415120210120B107417120210120BB9
:100A9A00437416120210120B5E7407120210120A25
:100AAA00F81202CB227452120210745812021074F5
:100ABA001412021074001202107415120210747FBC
:100ACA001202107417120210120B4374161202103B
:100ADA00120B5E740712021074AD1202101202CBCE
:100AEA0020B2FD7414120210747F12021022120A2C
:100AFA00352480120B071211C212021022B4F60317
:100B0A0024062250FB2212096A853A82853B83E534
:100B1A0082C4540FF9E583C46975F0028412021085
:100B2A002212096A853A82853B83E582C4540FF909
:100B3A00E583C46975F002842212094E85388285DC
:100B4A003983E582C4540FF9E583C46975F01184C9
:100B5A00120210221209E91202102274151202104E
:100B6A00120B107417120210120B43741612021091
:100B7A00120B5E740712021022120986853C8285C6
:100B8A003D83E582C4540FF9E583C46975F0028494
:100B9A0022120A3522300C08209205120B9BF548C6
:100BAA00E548B47711300B08754600754701C20B4A
:100BBA00120BE9D20A2250ED300A05754600C20A24
:100BCA00120BD0D20B2212031EE54693700B754608
:100BDA0000C20CC20D20B2FD22054612021022E507
:100BEA0047B40104120C0B22B40204120C2A22B4D8
:100BFA000304120C5222B40404120C7122120C9A2D
:100C0A0022120527E54693701175460074041202F4
:100C1A0010754702C20E20B2FD22054612021022AA
:100C2A002011061205B6020C36120637E5469370F5
:100C3A00117546007404120210754703C20E20B2E1
:100C4A00FD220546120210221206B8E546937011DB
:100C5A007546007404120210754704C20E20B2FDD4
:100C6A0022054612021022120739E54693701B75B7
:100C7A00460074061202107406120210740612025A
:100C8A0010754705C20E20B2FD2205461202102237
:100C9A002092151207BAE54693701A754600740633
:100CAA001202107406120210754701C20CC20DC25C
:100CBA000E20B2FD2205461202102212094E853874
:100CCA0082853983120DA7F53874311202107434F3
:100CDA00120210744A120210E53875F008841211D3
:100CEA0074120D5F120258744E12021074311202FD
:100CFA00107435120210744A120210E53875F008A1
:100D0A0084121174120D5F120258744E120210747A
:100D1A0034120210744A120210E538120D7D1202C2
:100D2A0058744E1202107435120210744A120210CC
:100D3A00E538120D65120258744E120210743612FA
:100D4A000210744A120210E538120D5F120258742A
:100D5A004E12021022F58275830022F52E752F009D
:0E0D6A00753207753300782E793212085686DE
:100D78008208868322F52E752F0075320775330099
:100D8800782E7932120856752E9F752F0F863208E5
:100D98008633782E7932120848868208868322E5BF
:100DA80082C4540FF9E583C469227438120210749E
:100DB8004A1202107440120D5F120258744E120249
:100DC800107430120210744A120210E53A120D5FC4
:100DD800120258744E120210227438120210744A09
:100DE80012021074C1120D5F120258744E120210D2
:100DF8007430120210744A120210E53A75F002A417
:100E0800120D5F120258744E120210227438120228
:100E180010744A12021074C0120D5F120258744EF8
:100E28001202107430120210744A120210E53A7558
:100E3800F0FFC5F0C395F075F002A4120D5F120221
:100E480058744E120210227438120210744A120298
:100E5800107403120D5F120258744E12021022749D
:100E680030120210744A1202107430120210744EBA
:100E78001202102212096A853A82853B83120DA755
:100E8800F53A7007120E4F1201B32279FFC9C399C0
:100E9800F53AB48003020EA65004120DE122120E98
:100EA8001422120986853C82853D83120DA7F53CE4
:100EB80075F00284120EC022B4020FD20F754E01D3
:100EC800754B00754C00754D002240EFC20FB408F9
:100ED8000D754E02754B0E754C08754D002240F18C
:100EE800B4100D754E03754B18754C0E754D0822D0
:100EF80040F1B4180D754E04754B20754C18754D9E
:100F08000E2240F1B41E0D754E05754B12754C0836
:100F1800754D002240F1B4250D754E06754B1675BA
:100F28004C08754D002240F1B42B0D754E07754BDA
:100F38000E754C06754D002240F1B4310D754E0802
:100F4800754B18754C0E754D062240F1B4370D756A
:100F58004E09754B12754C06754D002240F1B4418F
:100F68000D754E0A754B16754C06754D002240F1ED
:100F7800B44B0D754E0B754B14754C0A754D00220C
:100F880040F1B4540D754E0C754B10754C08754DE9
:100F9800002240F1B45D0D754E0D754B0C754C0675
:100FA800754D002240F1B4670D754E0E754B0E75E8
:100FB8004C0A754D002240F1B4700D754E0F754BFB
:100FC8000E754C04754D002240F1B47D0D754E1020
:100FD800754B14754C0E754D002240F1754E117508
:100FE8004B30754C18754D0022E549600C301205E0
:100FF80012100FC212121007221210D3D21222E5B9
:101008004EB54F0122F54F300F071210A0121024D1
:10101800221210431210621210812222743112021D
:10102800107431120210744A120210743312021032
:101038007430120210744E1202102274311202100F
:101048007431120210744A120210743112021074B0
:1010580030120210744E12021022743112021074EF
:1010680032120210744A12021074311202107430D3
:10107800120210744E1202102274311202107433CC
:10108800120210744A1202107431120210743012D3
:101098000210744E120210227431120210743212AD
:1010A8000210744A1202107430120210744E1202A6
:1010B8001074311202107433120210744A120210A2
:1010C8007430120210744E1202102274311202107F
:1010D8007431120210744A12021074301202107421
:0E10E8004E12021074311202107432120210F5
:1010F600744A1202107430120210744E12021074E6
:10110600311202107433120210744A120210743033
:10111600120210744E120210221211861203087463
:1011260031120210744A1202108E828F83120258F4
:10113600744E1202101211A6120308743212021013
:10114600744A1202108E828F83120258744E120253
:10115600101211B41203087433120210744A1202E8
:10116600108E828F83120258744E12021022B40F10
:1011760001224002740F22B4C00122400274C02230
:10118600C374C0954BF53EE54912117DB53E030289
:10119600119A4007E53E254BD21022254BC210225C
:1011A600201005E549254C22C3E53E254C2220109A
:1011B60005E549254D22C3E53E254D22C3B4FD0173
:1011C60022400374FD22C3B480012250027480229F
:1011D600B4F00122400274F022B478012240027475
:1011E6007822B43001224002743022C3B44701226F
:1011F6004002744722900010E004B410027400F01C
:10120600900000A98229F582E022900014E0FA906D
:101216000011E004B40F0274FFF09018A3932A9013
:101226000014F0900013E004B410027400F0F9907A
:101236000014E0FA900000E58229F582EAF0229097
:101246000014E0FA900012E004B4110274FFF0906A
:1012560018B2932A900014F0121229221211FB548C
:101266000160081211FB541F246022747F221211A0
:10127600FB75F02084221211FB75F01084221211E6
:10128600FB75F01F84228B878D0606BF8B8B0606A7
:10129600BE94800606BA899906BA8780BA06BB81CB
:1012A600C4BB06BB83A6818D069ABF06068D8780C2
:1012B6008D06BF838D8D060606060600BF838D8DBF
:1012C600068D87808D069ABF0606BB83A6818D068E
:1012D600BB81C4BB06BA8780BA06BA899906BE9492
:1012E600800606BF8B8B06068B878D0606A795A400
:1012F600060606060081B606AA818D069B8D05AAFE
:101306009691808D9606008B878D00BF8B8B00BED5
:10131600948000BA899900BA8780BA00BB81C4BBA1
:1013260000BB83A6818D009ABF008D87808D00BF8C
:10133600838D8D00809183A6818D008780008780B4
:1013460006848C00A000A00698060081BFBB008E14
:10135600A3008E89BF00AFA48EBF00838EBF009905
:1013660000C69183BDBE81C2009F82C4BE94898E91
:1013760081C200919AA79600A6848096008CC6A08A
:10138600BF9600949AB080A400C094838DBB8C81D4
:10139600BD818D009489AD89BF00B283A7899180F4
:1013A6008D0083088D07960FA580008C83B6808DEF
:1013B60000A781BBBF818C0083BF818CBB00A0BF0F
:1013C60094898DBB009906AA81BF00BB83BF819219
:1013D6008480BF009489C581BF00AA808C00BA9121
:1013E6008480008CA28D8D00A08D80A696BC00B254
:1013F600839183C4BB8000AA9184C21E0FB8A491B6
:101406001E0F009181BABF0689BA0600B280BF9846
:1014160000A7818DBF8106BB8780A7960600AE9484
:10142600878CBB00BBBF81C4BB00AA9ABB00BBBFF5
:1014360094818FBB00AB919A00BBBF89C7008CA07B
:10144600A781C200948706C3068D8D0694899106EE
:1014560000C78790C5068CA0A781C20600BF83C5BA
:0E1466008DA400AF828DBB068CA0A781C206AC
:1014740000C3898DA897BF00BF80BD97BF00BA8302
:101484008DC100B6A400C3888C81C200BFBB81B4E7
:10149400829482BFBB00AF9487C5BB00BB83C4BB2F
:1014A400008C81BBBF968000C7A3960083949900EB
:1014B400AE94808C00BB848E8EBDB687808D8D00EB
:1014C400BA91A39600A689BF9400949A8D8D00A426
:1014D400BCBC818D8D00C392A3C100BBC3878000B7
:1014E400A69791B000A6888EAE96BA8A8A9200B268
:1014F400969100A68B8C818D00919AAE8000AB9C56
:10150400008C83838D8D009484BBBF848C878D0075
:10151400BB81BBBF9600AA9487A796008C87A79629
:1015240000BA87A796009281C6BC008780BB00B72B
:101534009600AB87AE8000A406C29A009EBB008EC4
:10154400A400AEA38E0084B5009183BABF00948733
:1015540080BF00BF86948D00888E0088BA00878D76
:10156400AE9600818E00B89500A6948890008D8771
:1015740080BB00C38B8B9100BBBF998C8000BA9455
:101584008000A492BF00BF89C50681ABA3BF06003B
:10159400C69180A70084809104AA8004AA82C4050D
:1015A40000BE838FC506A00600878000A000BF99F7
:1015B4008D9AAFA4BB008CC6A0BF96BB008C848F51
:1015C400C280BB009489AD89BFBB009FA681BB00CC
:1015D4008EA4AB85AE8000BBC38780A699C296005B
:1015E400B387BF00918ABB81BA96008C8484848CB3
:1015F40000BBAC8480AE968C838D00A78106BF9718
:101604008C818D9ABF940500A781068C98BBBF96E8
:1016140088BAA08D8106A696A706008C81BBBF96CA
:10162400C69483A780AE828EBF00BF89C50581ABF7
:10163400A3BF0500AB919A00B3A405BF8B05BE817F
:101644000500BBBF89C7009187BABA00BA8480BFBE
:1016540081B29A8DBBBF0500BB8C9F06918480C468
:101664000600BB97B600AE94808C0688BA0600B715
:101674009ABF00AA819180BA06818E0600AE83BB10
:10168400BF949C00A6948480AE0588BA0500AA94F1
:101694009AC405BE948B0500918AC40583BF0500D6
:1016A400C2819200BF89C5BB0581ABA3BF0500AB56
:1016B400919ABB00B3A4BB05BF8B05BE810500BBDB
:1016C400BF89C7BB009187BABABB00BA8480BFBBCD
:1016D40081B29A8DBBBF0500BB8C9FBB06918480F1
:1016E400C40600BB97B680BB00AE94808CBB068852
:1016F400BA0600B79ABFBB00AA819180BABB068123
:101704008E0600AE83BBBF949CBB00A6948480AEBF
:10171400BB0588BA0500AA949AC4BB05BE948BBBCA
:101724000500918AC4BB0583BF0500C28192BB003A
:10173400818DC29482AF81AA8191008D8780BB0084
:10174400C38B8B9100BA948000BA9AAA9F81BB0084
:10175400A6888EAE96BA8A8A9200BBBF998C800006
:10176400AF98C500BA848FC280008C81BBBF800053
:10177400AE838C8DBF008C8480AE8000AE828C8161
:10178400BFB6C200AE9A8DA89586BB00C087C5A718
:1017940081C4008C99AE9686BB00AF9487C5BB000C
:1017A400BFBB81B4829482BFBB00BC81BF80059162
:1017B4008780BF800500C2949AA780B899BB81BB7B
:1017C40000B2839183C4BB8000B280BF98BB00BACF
:1017D40091A396BB00C78790C5058CA0A781C205BD
:0E17E40000AA9183C506AF89C506BB00A78188
:1017F2008DBF8106BB8780A796BB00AA949A8DBB3A
:1018020000AA818E828E84BB00BA9ABB81BB00C3C0
:1018120092A3C100AF828DBB068CA0A781C2060035
:10182200BF80BD97BFBB00AA8006C299A7060083EE
:101832008EBF00990600878005AFA48EBF058EA4D7
:101842000500060606838D80939A060606000606A4
:101852008480048C808E06060006A406C29A0606C0
:1018620000AA80BB8480B1BB060600BBA40600A60A
:101872009F060600918480C40600AB86BF060082E4
:10188200C4BFB69F800600A684809F00A689BF04BD
:1018920082A696048C838D0606008E9A8C91800611
:1018A2000003002C0C01057E2133E6FF0B4D68146A
:1018B2006405140D004B1A26351E1A96114042C8B3
:1018C200C921232527292C2E3134373A3E41454957
:1018D2004E52575D62686E757B838B939CA5AFB940
:1018E200C4D0DCE9F7F700000000000000010002AC
:1018F20000030004000500060006000700070008B8
:10190200000800090009000A000A000B000C000C84
:10191200000D000E000F0010001100120013001441
:10192200001600170018001A001C001D001F0021DD
:101932000023002500270029002C002E003100344E
:101942000037003A003E004100450049004E005277
:101952000057005C00630068006E0075007C008325
:10196200008B0093009C00A500AF00B900C400D01A
:1019720000DC00E900F70106011501260137014AE2
:10198200015D01720188019F01B801D201EE020BD3
:10199200022A024B026E029302BA02E40310033FD0
:1019A200037003A403DC04170455049704DD052720
:1019B200057505C80620067D06E0074907B8082D0B
:1019C20008A9092D09B90A4D0AB00B900C400CFA6E
:1019D2000DC00E910F6F0F6F464C414D4520544183
:1019E2004C4B494E472D53594E54482D4D4F44555B
:1019F2004C45204555524F205241434B20564552AB
:101A020053494F4E202D203230313120564552530A
:101A1200494F4E20312E30302028632962792061CF
:051A22006D70657265A6
:00000001FF
